:100000000C9446030C948D030C948D030C948D0377
:100010000C948D030C948D030C948D030C948D0320
:100020000C948D030C948D030C94CD210C94892198
:100030000C948E280C948D030C948D030C948D03DA
:100040000C948D030C948D030C948D030C948D03F0
:100050000C948D030C946A280C948D030C948D03DE
:100060000C948D030C948D030C948D030C948D03D0
:100070000C948D030C948D030C948D030C948D03C0
:100080000C948D030C948D030C948D030C948D03B0
:100090000C948D030C948D030C948D030C948D03A0
:1000A0000C948D030C948D030C948D0305010902AF
:1000B000A10185020901A100050919012905150001
:1000C00025019505750181029501750381010501E1
:1000D000093009311581257F950275088106093897
:1000E0001581257F950175088106050C0A380215D2
:1000F00081257F950175088106C0C005010980A191
:1001000001850319012AB700150126B7009501756D
:10011000108100C0050C0901A101850419012AA064
:1001200002150126A002950175108100C005010984
:1001300006A1018505050719E029E71500250195A8
:1001400008750181020507190029EF1500250195A1
:10015000F0750181020508190129059505750191C0
:1001600002950175039101C00660FF0961A10109B3
:1001700062150026FF0095207508810209631500AD
:1001800026FF00952075089102C005010906A1010E
:10019000050719E029E71500250195087501810279
:1001A0009501750881010507190029FF150026FF33
:1001B0000095067508810005081901290595057542
:1001C000019102950175039101C00000000000003B
:1001D000000000000000000000000000000000001F
:1001E00000000000000000000000000000007E0F82
:1001F00000D4FFFFFFC700000078000000000000EF
:1002000000002A2B28000000000000000000000071
:10021000000000000029000000002C1E34202122D4
:1002200024342627252E362D3738271E1F2021223D
:10023000232425263333362E37381F0405060708B6
:10024000090A0B0C0D0E0F101112131415161718A6
:10025000191A1B1C1D2F3130232D350405060708E4
:10026000090A0B0C0D0E0F10111213141516171886
:10027000191A1B1C1D2F3130354C000101010101E1
:10028000010101010202020202020202020303034F
:10029000030303030304040404040404050505051F
:1002A00005060606060607070707070808080809DF
:1002B0000909090A0A0A0B0B0B0C0C0C0D0D0D0E8B
:1002C0000E0E0F0F0F101011111112121313141420
:1002D000151516161717181819191A1A1B1B1C1D95
:1002E0001D1E1E1F202021222223242425262627EE
:1002F0002829292A2B2C2D2D2E2F30313232333420
:1003000035363738393A3B3C3D3E3F404142434425
:1003100045464748494A4C4D4E4F50515354555607
:1003200058595A5B5D5E5F616264656668696B6CB3
:100330006D6F7072737577787A7B7D7E808283852E
:1003400087888A8C8E8F91939596989A9C9EA0A26E
:10035000A3A5A7A9ABADAFB1B3B5B7BABCBEC0C278
:10036000C4C6C9CBCDCFD1D4D6D8DBDDDFE2E4E73C
:10037000E9EBEEF0F3F5F8FAFDFFFFAA7F55402216
:1003800023252628292A2C2D2F3032333536383A8A
:100390003B3D3E4042434547494A4C4E50515355E0
:1003A00057595A5C5E6062646668696B6D6F717301
:1003B0007577797B7D7F81838587898A8C8E909202
:1003C0009496989A9C9E9FA1A3A5A7A8AAACAEAF0D
:1003D000B1B3B4B6B8B9BBBCBEBFC1C2C3C5C6C752
:1003E000C9CACBCCCDCED0D1D2D2D3D4D5D6D7D703
:1003F000D8D9D9DADADBDBDBDCDCDCDCDCDDDDDD4B
:10040000DDDCDCDCDCDCDBDBDBDADAD9D9D8D7D746
:10041000D6D5D4D3D2D2D1D0CECDCCCBCAC9C7C6F3
:10042000C5C3C2C1BFBEBCBBB9B8B6B4B3B1AFAE31
:10043000ACAAA8A7A5A3A19F9E9C9A9896949290D7
:100440008E8C8A89878583817F7D7B7977757371AF
:100450006F6D6B6968666462605E5C5A595755538C
:1004600051504E4C4A4947454342403E3D3B3A3845
:1004700036353332302F2D2C2A29282625232229C0
:10048000003A003B003C003D003E003F0040004180
:10049000004200430044004500C35C490035001E93
:1004A000001F002000210022002300240025002638
:1004B0000027002D002E002A004D002B0014001AEA
:1004C000000800150017001C0018000C0012001393
:1004D000002F00300031004C0039000400160007E6
:1004E0000009000A000B000D000E000F003300345D
:1004F00000280000000000E10000001D001B0006B5
:10050000001900050011001000360037003800E522
:100510000052000000E000E300E2000000000000E4
:10052000002C0000000000E600E400500051004FE5
:10053000000000005C010001000100010001000159
:1005400000010001000100010001000100010001A3
:100550000001000100010001000100010001000193
:100560000001000100010001000100010001000183
:100570000001000100010001000100010001000173
:100580000001000100010001000100010001000163
:100590000001000100010001000100010001000153
:1005A0000001000100010000000000010000000146
:1005B0000001000100010001000100010001000133
:1005C0000001000100C35C00000100010001000007
:1005D000000000000001000000000001000100C058
:1005E0005CC25C010000001E0F0500047F3F1F6419
:1005F0003214643214783C1E1E140A0509025B0092
:10060000030100A0FA09040000010301010009210F
:10061000110100012240000705810308000A0904B6
:100620000100020300000009211101000122220043
:1006300007058203200001070503032000010904C8
:100640000200010300000009211101000122BC0089
:100650000705840320000A1201100100000008545D
:100660004D07200100010203010403300000000EC9
:100670000345003700350048004F005400000006D5
:10068000034D0054000000040309040011241FBEA0
:10069000CFEFDAE0DEBFCDBF04B603FE27C0809106
:1006A000A9049091AA04A091AB04B091AC04873046
:1006B000904BA740B04BD1F41092A9041092AA0419
:1006C0001092AB041092AC0414BE84B7877F84BF31
:1006D0000FB6F894A89580916000886180936000BF
:1006E000109260000FBEE0E0F8E3099524E0AEE967
:1006F000B1E001C01D92A93AB207E1F711E0A0E014
:10070000B1E0E8E0F5E502C005900D92AE39B10721
:10071000D9F70E94A4220C94372A0C940000E8ED2B
:10072000F0E080818E7F80831092E2001092DA00E8
:100730001092E100A0EEB0E08C9181608C938081FA
:100740008F77808319BCA7EDB0E08C918E7F8C935E
:1007500080818F7E80831092730408952091E4003D
:100760003091E50095E6A9012091EC00822F81707F
:1007700020FF06C08091E80080FF06C080E0089559
:100780002091E80022FD1AC080919804882389F006
:10079000853089F08091EB0085FD0FC02091E40049
:1007A0003091E50042175307F9F29150E1F684E0E9
:1007B000089582E0089583E0089581E00895EF921E
:1007C000FF920F931F93CF937C018B010E94AE0386
:1007D000C82F811117C08091E80085FD0BC0809162
:1007E000E8008E778093E8000E94AE03882399F397
:1007F000C82F08C0F70181917F018093F10001505B
:10080000110949F78C2FCF911F910F91FF90EF9015
:10081000089580919A0487FF13C08091E80082FFB9
:1008200006C08091E8008B778093E80004C0809137
:1008300098048111F2CF0895809198048823D9F308
:100840008091E80080FFF8CF8091E8008E77ECCFB0
:10085000982F9093E900242F762F50E0891731F0DC
:100860007091EC002091ED005091F00021FD07C047
:100870009F5F973071F78093E90081E00895309190
:10088000EB003E7F3093EB003091ED003D7F3093E5
:10089000ED003091EB0031603093EB007093EC0091
:1008A0002093ED005093F0002091EE0027FDE0CF63
:1008B00080E00895CF92DF92EF92FF920F931F9303
:1008C000CF93DF93C8EDD0E088818F7E8883E7EDFA
:1008D000F0E080818160808384E082BF81E080934A
:1008E000730488818E7F888302EE10E0F801108205
:1008F0001092DA0081EEC82ED12CF6011082888188
:100900008F77888388818068888388818F7D8883BA
:1009100019BC1092980410929904109297041092A6
:10092000960490EEE92EF12CF70180818B7F808375
:1009300088818160888342E060E080E00E94280432
:10094000F60180818E7F8083F801808181608083C1
:10095000808188608083F70180818E7F8083888199
:1009600080618883DF91CF911F910F91FF90EF906D
:10097000DF90CF900895FC018091A0049091A10494
:1009800086179707A0F06115710529F49091E8008A
:100990009E779093E80090E06115710551F49111F4
:1009A00008C08091E80082FF34C080E00895BC0157
:1009B000F2CF809198048823C1F18530C1F18091F4
:1009C000E80083FD30C08091E80082FDEACF80918D
:1009D000E80080FFE1CF8091F3002091F200382FF2
:1009E0006115710519F02830310558F091E0283073
:1009F000310509F090E02091E8002E772093E8007F
:100A0000CBCF81918093F100615071092F5F3F4FEF
:100A1000E7CF80919804882341F0853041F08091A0
:100A2000E80083FFBECF81E0089582E0089583E06F
:100A30000895089580E008958091750408959C01BB
:100A40004FB7F89480916F0490917004A091710455
:100A5000B09172044FBF821B930B08952FB7F89487
:100A600080916F0490917004A0917104B091720410
:100A70002FBF0895809124048111109224040895B9
:100A80008091230490912204892B90912104892B39
:100A90008093A001909124049923A1F0892B809345
:100AA000A00180911C01882341F18091350487FFCA
:100AB00024C08EE1E2EAF1E090E0815000F591116E
:100AC0000E943A05E0913804F09139043097E1F042
:100AD00080911C01882359F08091350487FF07C05D
:100AE0008091A0018093A10185E08093A001028004
:100AF000F381E02D80EA91E0099486E0DBCF21913B
:100B00002223D9F29F5FD9CF089590911C01992398
:100B1000D1F09091350497FF16C0E82FE695E69541
:100B2000E695EE31E0F4F0E0E056FE4F282F277016
:100B300081E090E001C0880F2A95EAF780959281C4
:100B4000892382830895E2EAF1E09191891303C039
:100B5000DF0111971C9291E0E83AF907B1F7089587
:100B600090911C019923C1F09091350497FF14C016
:100B7000E82FE695E695E695EE31F8F4F0E0E056DC
:100B8000FE4F877021E030E001C0220F8A95EAF71E
:100B90008281822B82830895A2EAB1E0EFEF90E098
:100BA0002D91821751F0EF3F19F4211101C0E92F67
:100BB0009F5F9630A9F7EF3F09F408950E2E000CC1
:100BC000FF0BE056FE4FE6CF2FE0929F800D1124E1
:100BD000982F977086958695869525E0829FF001DF
:100BE0001124EC51FC4F50E040E080E0219130E0D6
:100BF000092E02C0369527950A94E2F72170332713
:100C0000042E01C0220F0A94EAF7822B4F5F5F4F38
:100C10004530510559F708952FE0929F800D11241A
:100C2000982F977041E001C0440F9A95EAF7869596
:100C30008695869595E0899FF0011124EC51FC4F33
:100C400090E080E070E05191DF0111979B01082E48
:100C500002C0369527950A94E2F721702195252741
:100C6000242325272C9301968530910561F708955B
:100C70008091E3039091B203981301C008958F5FB0
:100C80008770FACF882341F08095909123048923BF
:100C9000809323040C9440050895882339F09091A3
:100CA0002304982B909323040C94400508952091DD
:100CB000A8033091A9032817390771F09093A9036D
:100CC0008093A803E0913804F0913904309721F023
:100CD0000084F185E02D099408952091A6033091B8
:100CE000A7032817390771F09093A7038093A603F1
:100CF000E0913804F0913904309721F00680F781B3
:100D0000E02D09940895E0913804F091390430976A
:100D100021F00190F081E02D099480E00895CF92B8
:100D2000DF92EF92FF92843030F5811125C09091CF
:100D300080009F7D909380002E98282F30E0AFEFA9
:100D4000BFEF0E94282A23E030E040E050E00E94FC
:100D5000062AC9012C3764E13607A0F469E070E087
:100D60000E94DF2870938B0060938A00FF90EF90C1
:100D7000DF90CF90089583E09091800090629093EF
:100D80008000DBCF2A50374D4F4F5F4F942F832F7A
:100D9000722F662725EF38E241E050E00E94062AD4
:100DA00069017A01CA01B9010E94B5289B01AC0111
:100DB000C701B6010E94B528672F782F892F992780
:100DC0006115710521E08207910561F66FEF7FEFF4
:100DD000C9CF282F220F220F220F90915B0497700A
:100DE000922B90935B04987F21E009F420E090918E
:100DF0005B0420FB90F990935B040C948F06FA013E
:100E0000811101C0FB01099480915E04982F9E7F9F
:100E100061F48170826080935E0480916104833309
:100E200018F082E38093610408958635B0F38170F1
:100E30008465F1CFAF92BF92DF92EF92FF920F9352
:100E40001F93CF93DF93182F062FE901433308F048
:100E500042E3E42FF0E0E658FD4F011110C0E491A9
:100E60005E2F4E2F4983E8835A83DF91CF911F91E4
:100E70000F91FF90EF90DF90BF90AF900895202FDB
:100E800030E04491D42EE42EF12C56E0159FC001A1
:100E90001124EFEFF0E0BF010E94DF28812F90E0E6
:100EA000880F991F55E5569FD001579FB00D11240B
:100EB0008A1B9B0B982F990F890F5F01A21AB30A07
:100EC000AE9CD001AF9CB00DBE9CB00D11245B2F29
:100ED000089F80011124012F11275F01A01AB10A78
:100EE000AE9C8001AF9C100DBE9C100D11245F01C3
:100EF000A81AB108A29EC001A39E900DB29E900DAB
:100F00001124892F9927E81BF90BEE9DC001EF9D55
:100F1000900DFE9D900D1124E92F62307105A1F016
:100F200050F46115710509F49DCF6130710581F0B0
:100F3000EB2F512F97CF6430710569F080F0663048
:100F4000710509F48FCFF4CFE42F4B2F592F8ACF9F
:100F5000E42F412F87CFEB2F542F492F83CF4B2FD7
:100F60005D2DE12F7FCF0E942E059C0190914904B9
:100F700080914A04982B21F0309346042093450435
:100F800090914B0480914C04982B21F030934304B2
:100F900020934204E0913804F0913904309749F0ED
:100FA00082E0809347040480F581E02D87E494E09B
:100FB0000994089590E080E00E946D0690E080E042
:100FC0000E94570610922204109221040E944005AC
:100FD00086E0E7E4F4E0DF011D928A95E9F71092DC
:100FE0004404109241041092AB030C94B307609335
:100FF000A5047093A6048093A7049093A8040C946E
:10100000DA070F931F936091A5047091A604809155
:10101000A7049091A8048B019C0106701127222738
:101020003327063011052105310529F468601F9129
:101030000F910C94F707677FFACF0F931F9341E04E
:1010400050E060E070E004C0440F551F661F771F3A
:101050008A95D2F7CB01BA016095709580959095ED
:101060000091A5041091A6042091A7043091A80432
:1010700060237123822393231F910F910C94F70710
:10108000909120048095892380932004282F277035
:1010900071F4282F082E000C330B9217130639F029
:1010A0008595859585950E941D08109220040895C8
:1010B0000F931F9341E050E060E070E004C0440FE4
:1010C000551F661F771F8A95D2F78091A5049091CE
:1010D000A604A091A704B091A8048A019B01082B43
:1010E000192B2A2B3B2BC901B8011F910F910C948E
:1010F000F707609325047093260480932704909348
:1011000028040C94DA0790914904803F59F48091A7
:101110004A0487FF0DC010924A0491110BC010922F
:10112000440408C0813F81F480914A0418169CF35E
:10113000992381F080914B0490914C04892B09F004
:1011400064C0109241040895823F49F497FFF0CFA4
:101150001092490480914A048111ECCFE0CF833F83
:1011600019F41916ACF3E4CF20914B04893F29F40C
:101170001216F4F610924B04DBCF8A3F19F427FFC6
:10118000D7CFF8CF20914C048B3F29F427FFD0CF45
:1011900010924C04CDCF8C3F19F41216CCF3C8CF6B
:1011A000843F31F4809148048E7F80934804C0CFFF
:1011B000853F21F4809148048D7FF7CF863F21F44D
:1011C000809148048B7FF1CF873F21F480914804C0
:1011D000877FEBCF883F21F4809148048F7EE5CF55
:1011E0008D3F31F48091AB038E7F8093AB03A0CF12
:1011F0008E3F21F48091AB038D7FF7CF8F3F09F0B5
:1012000097CF8091AB038B7FF0CF0895882309F4AB
:1012100059C0823871F40E94830681FF53C089E36C
:101220000E94B0050E94400589E30E9485050C9448
:101230004005833859F40E94830680FF43C083E54C
:101240000E94B0050E94400583E5EFCF843859F431
:101250000E94830682FF36C087E40E94B0050E9488
:10126000400587E4E2CF9CEF980F913AF0F290E2CC
:10127000980F983088F4877021E030E0A90102C00F
:10128000440F551F8A95E2F7CA0180959091230477
:10129000892380932304CBCF9BE5980F933020F4D0
:1012A00090E080E00C946D0698E5980F973120F45B
:1012B00090E080E00C945706803F20F00E94830865
:1012C0000C94B30708958091AB0380FD16C081FD97
:1012D00016C082FD16C0809141048823A1F0883297
:1012E00080F428E0829FC001112468E270E00E942F
:1012F000F328862F672B39F0089582E0089584E063
:10130000089588E0089581E008958091AB0380FD01
:1013100014C081FD14C082FD16C08091440488234E
:1013200081F0843180F422E3829FC001112464E1C2
:1013300070E00E94F328862F08958CE0089589E1DB
:10134000089585E0089582E30895803F31F40E9476
:101350008509819580934A040895813F19F40E947C
:101360008509F8CF823F31F40E94850981958093E9
:1013700049040895833F19F40E948509F8CF893FF5
:1013800029F40E94630980934B0408958A3F21F455
:101390000E9463098195F7CF8B3F31F40E94630966
:1013A000819580934C0408958C3F19F40E94630941
:1013B000F8CF843F31F480914804816080934804E1
:1013C0000895853F21F4809148048260F7CF863FDD
:1013D00021F4809148048460F1CF873F21F480910B
:1013E00048048860EBCF883F21F4809148048061F5
:1013F000E5CF8D3F31F48091AB0381608093AB03E7
:1014000008958E3F21F48091AB038260F7CF8F3F28
:10141000B9F78091AB038460F1CFF894E82FE2959F
:10142000EF70F0E031A1282F2F7081E090E001C033
:10143000880F2A95EAF7982F9095932391A392A16C
:10144000892B82A3789408959091350492FF06C069
:10145000282F28712830F9F4877F846093FF06C015
:10146000282F28712831F1F4877E84612091360479
:1014700020FF06C0382F38713830D9F4877F81605B
:1014800021FF06C0282F28712831D1F4877E816181
:1014900094FD877E0895282F24712430F9F68B7FE0
:1014A0008860DCCF282F2471243101F78B7E88617E
:1014B000DDCF382F3171313019F78E7F8860E0CF62
:1014C000282F2171213121F78E7E8861E1CF81FDA6
:1014D00002C0479A089547980895CF9384E090E01A
:1014E0000E948C29C82F81E290E00E948C29982FBD
:1014F0008C2FCF9108950F931F93CF93DF93843058
:1015000030F5663020F54F3010F5C42FD0E0CC0F09
:10151000DD1F2EE1629FC00DD11D112434EB839F8E
:10152000C00DD11D1124CE0186960E948C29082F52
:1015300010E0102F0027CE0187960E948C29980179
:10154000282BC901DF91CF911F910F91089590E051
:1015500080E0F8CF462F843038F4763028F46F30AE
:1015600018F4672F0C947B0A90E080E00895CF93E5
:10157000DF930E94AA0AEC0182389105A9F1D8F5FF
:101580008133910509F496C048F58932910509F433
:101590008AC08A9709F495C0C11521E5D20708F0E1
:1015A000BCC0C11530E5D30708F014C1C83ED10551
:1015B00008F09CC0C03ED10560F5C83AD10508F0DE
:1015C00087C0C53AD10508F0FDC0C130D10509F189
:1015D0002097F9F0C430D105E0F440C0853391057F
:1015E00009F45AC0C997C1F680913504837089F017
:1015F000C0EED0E00EC0833E910599F170F4803EBC
:10160000910501F1823E910539F68091350482FD04
:1016100021C0CE01DF91CF910895863E910561F101
:10162000873E910571F1843E910509F0B5CF809117
:10163000360481FFEECF80913504C7EED0E084FD03
:101640000DC0E7CF8091350480FD12C19091360422
:1016500090FFDFCFC3EED0E084FFDBCFD0E0C0E06F
:10166000D8CF8091350482FD06C19091360490FD5B
:10167000BFCF84FFCECFF2CF8091350483FDDDCF85
:10168000C8CF8091350483FDF9C09091360491FF55
:10169000F0CFC4EED0E0BDCF8091350485FFB9CF47
:1016A000C9E2D0E0B6CF8091350485FFB2CFC5E363
:1016B000D0E0AFCF8091350486FFABCFCAE2D0E057
:1016C000A8CF8091350486FFA4CFC1E3D0E0A1CF9D
:1016D000CF3BD10518F6C85AD0E0CC0FDD1FC55B53
:1016E000DE4F0990D881C02DD46493CFC11540E25C
:1016F000D40758F4C11581E0D80708F08ACFC03F5D
:10170000D10508F4ABCFD06584CFC11590E4D907DB
:1017100008F4A4CFDF70D06A7CCFC11525E5D207CD
:1017200000F5C11534E5D30708F08AC0C11543E5BB
:10173000D40708F071C0C11582E5D80708F467C066
:10174000CE018370992721E030E002C0220F331FC1
:101750008A95E2F7C695C69580E2C89FE0011124FC
:1017600052C0C11599E5D907A8F4C11528E5D207DB
:1017700008F06BC0C11536E5D30708F06FCF8C2F8A
:101780000E94240AC82FD0E0DC2FCC27CC27DF71A1
:10179000D0623FCFC1154AE5D40708F45BC0CE0143
:1017A00090568115904208F059CF8D2F8F710E946D
:1017B000240A90E0982F882788279F719C012C2B62
:1017C000E901E6CFC55AD0E0C85BDE4FC881D0E062
:1017D000D0641FCFCE01E4E096958795EA95E1F7B6
:1017E00083702C2F26952695237040E2249F90012C
:1017F0001124382B8C2F8370C1E0D0E002C0CC0FB5
:10180000DD1F8A95E2F7C22BD32BDC6802CFDC2FD9
:10181000CC27C16FD06AFDCECE018370992721E01D
:1018200030E002C0220F331F8A95E2F7C695C695B5
:1018300090E2C99FE0011124C22BD32BDA68E9CED4
:10184000DC2FCC27C46FD06AE4CEDC2FCC27C06F4E
:10185000D06ADFCE8C2F8F700E94240A34E0D69598
:10186000C7953A95E1F7CF709C2FEC01D069D1CEA6
:10187000C9E3D0E0CECEC2EED0E0CBCEC6EED0E013
:10188000C8CEBF92CF92DF92EF92FF920F931F9339
:10189000CF93DF938C01C090A504D090A604E09074
:1018A000A704F090A8048091250490912604A091AB
:1018B0002704B0912804C82AD92AEA2AFB2ACFE1B2
:1018C000D0E0BC2ED701C6010C2E04C0B695A7955A
:1018D000979587950A94D2F780FD0EC0219788F7D7
:1018E000B12C8B2DDF91CF911F910F91FF90EF9035
:1018F000DF90CF90BF900895B8018C2F0E94B70A57
:10190000019761F3EECFCF93DF93EC010E94410C7E
:10191000BE01DF91CF910C94B70A0E94830C292F4E
:101920002F7092959F7092509E3078F4E92FF0E0DE
:10193000E75CF54D0C940729803F19F020F4883EB0
:1019400020F481E00895843FE1F380E00895883E2B
:10195000C0F3813FD1F7F5CF822F86958695869586
:101960000895682F86E090E00C94A029CF93DF9330
:10197000C6EFD2E060E0CE010E94A0292196C115F9
:1019800084E0D807B9F7DF91CF9108951F93CF93E3
:10199000DF93122F8430F8F46630E8F44F30D8F437
:1019A000C42FD0E0CC0FDD1F9EE1699FC00DD11D7B
:1019B000112494EB899FC00DD11D1124632FCE01FA
:1019C00086960E94A029612FCE018796DF91CF9144
:1019D0001F910C94A029DF91CF911F910895AF9290
:1019E000BF92CF92DF92EF92FF921F93CF93DF933C
:1019F0008FE7C82E84E0D82ED0E07601C0E014C076
:101A0000F50125913491412F6C2F8D2F0E94C60C2A
:101A100082E0A80EB11C1F5F1F3091F78EE1E80E27
:101A2000F11CCF5FC63019F0570110E0E9CFDF5F3E
:101A300084EBC80ED11CD43001F7DF91CF911F91F8
:101A4000FF90EF90DF90CF90BF90AF900895CF932D
:101A5000DF9300D00F92CDB7DEB790919804943009
:101A600011F589837B836A839093E9008FEF9091CE
:101A7000E800815095FD06C095ED9A95F1F70000BC
:101A80008111F5CF8091E80085FF0DC050E040E066
:101A900063E070E0CE0101960E94DF038091E800D0
:101AA0008E778093E8000F900F900F90DF91CF9189
:101AB0000895BC0184E00C94270DBC0183E00C94D4
:101AC000270D9C0184E08093E9009FEF8091E8005E
:101AD000915085FD06C085ED8A95F1F700009111C2
:101AE000F5CF8091E80085FF0CC050E040E066E053
:101AF00070E0C9010E94DF038091E8008E77809337
:101B0000E8000895CF93DF93EC0180911C018823B6
:101B1000B1F18091350487FF32C060E284E08093A8
:101B2000E9008FEF9091E800815095FD06C095ED9A
:101B30009A95F1F700008111F5CF8091E80085FFBB
:101B40001BC080911C0170E050E040E0811104C096
:101B500050E040E068E070E0CE010E94DF03809139
:101B6000E8008E778093E80080E2FE01A6E7B4E00B
:101B700001900D928A95E1F7DF91CF91089568E089
:101B800081E0CDCF81E08093E00080E28093D800B7
:101B90001092C9008FE19EE40197F1F700C00000A8
:101BA00087E090EBDC018093A9049093AA04A093B2
:101BB000AB04B093AC0488E19CE00FB6F894A89510
:101BC000809360000FBE90936000FFCFCF93C82F2B
:101BD000882309F4AEC08238C1F40E94830681FDD7
:101BE000A8C089E30E94B0050E9440052FEF81EE56
:101BF00094E0215080409040E1F700C0000089E36C
:101C00000E948505CF910C9440058338A1F40E9471
:101C1000830680FD8EC083E50E94B0050E944005CA
:101C20002FEF81EE94E0215080409040E1F700C01A
:101C3000000083E5E5CF8438A1F40E94830682FD8D
:101C400078C087E40E94B0050E9440052FEF81EE26
:101C500094E0215080409040E1F700C0000087E40C
:101C6000CFCF8CEF8C0F813A88F580911C018823AF
:101C700001F18091350487FF1CC0EC2FE695E695B5
:101C8000E695F0E0E056FE4F828190E04C2F4770E1
:101C900021E030E002C0220F331F4A95E2F7822391
:101CA0009323892B79F08C2F0E9485050E94400593
:101CB00009C0E2EAF1E08191C817A9F321E0E83A0E
:101CC000F207C9F78C2F0E94B0059CCF80E28C0FE1
:101CD000883068F4C77021E030E001C0220FCA9557
:101CE000EAF780912304822B809323048BCFEBE5CA
:101CF000EC0FE33040F4F0E0E85BFE4F808190E0D1
:101D0000CF910C946D06E8E5EC0FE73150F4F0E06C
:101D1000EE0FFF1FE55BFE4F80819181CF910C9408
:101D20005706C03F30F08C2F0E94A509CF910C942C
:101D3000B307CF9108951F93CF93DF93182FD0E06F
:101D4000C0E0893311F4C0E5D0E0812F0E94E60D98
:101D5000209731F4812FDF91CF911F910C940609C8
:101D60008FE99FE00197F1F700C000002197F0CFC5
:101D70000F931F93CF93DF93C62FD42F022FFC0115
:101D800082818823A1F06093A4040E942E05909381
:101D9000A3048093A204C77081E001C0880FCA9594
:101DA000EAF7DF91CF911F910F910C944D0680912E
:101DB000A404681335C08091A2049091A3040E94EA
:101DC0001F05883C910560F510E21D0FCD17B9F095
:101DD00080E28C0F883040F4C77081E001C0880F2A
:101DE000CA95EAF70E944206183048F481E09D2F18
:101DF000977001C0880F9A95EAF70E944D06802FD0
:101E00000E949B0E183098F4D77081E001C0880FB3
:101E1000DA95EAF7DF91CF911F910F910C9442066A
:101E2000C77081E001C0880FCA95EAF7F3CFDF9150
:101E3000CF911F910F91089580915E0480FD0AC09B
:101E4000E6ECF1E0118210821282339652E0EA371A
:101E5000F507C1F76A9A3EB13B7F2EB124604FB7B8
:101E6000F89486EC91E0FC015191CF0168E02EB925
:101E7000000000C057FF3EB9550F000000C000C071
:101E800000C03EB900C06A9591F7F2E08A379F071B
:101E900051F74FBF8FE594E00197F1F700C00000C4
:101EA0000895EF92FF921F93CF93DF93EC0186EC9E
:101EB000E82E81E0F82E10E08C81970140916104BA
:101EC00060916004810F0E941A071C5F83E0E80E96
:101ED000F11C103F89F70E941C0F9A818C8190FFA2
:101EE00008C08F5F8C83DF91CF911F91FF90EF909F
:101EF00008958150F7CFBF92CF92DF92EF92FF9279
:101F00000F931F93CF93DF93FC018281DD24DA943A
:101F100080FD02C0DD24D39406EC11E0D0E0C0E0E7
:101F20002CE3B22EF80111821082128294E0E92E85
:101F3000F12CC12C8091C3018C0D8D330CF43DC06C
:101F40006B2D0E94D128892F082E000C990B8C171D
:101F50009D0791F4809161048E9DA0018F9D500D8D
:101F600011245595479555954795980160916004C2
:101F700080915F040E941A07CD0CF1E0EF1AF1087E
:101F8000C9F621960D5F1F4FCC33D10559F60E943B
:101F90001C0F8091C30191E0D91215C0811111C0AD
:101FA0008BE38093C301DF91CF911F910F91FF903D
:101FB000EF90DF90CF90BF90089587FFC5CF845CEE
:101FC000C3CF8150EECF90E00196BE010E94F3286E
:101FD000E8CF0F931F93CF93DF93C6ECD1E0FE01C0
:101FE000118210821282339682E0EA37F807C1F735
:101FF00010E000E08091C401082E000C990B081736
:1020000019078CF180911001082E000C990B801794
:1020100091074CF19E0140916104609160048091B0
:102020005F040E941A070F5F1F4F23960C331105A0
:1020300009F70E941C0F80910F019091C401980F25
:102040009093C40120911001280F209310011216C3
:1020500014F49B331CF0819580930F01DF91CF9195
:102060001F910F910895198218821A82DCCF8F92E6
:102070009F92AF92BF92CF92DF92EF92FF920F9317
:102080001F93CF93DF93EC014C81042F10E0980154
:10209000D8010E94282A9B01AC010E94F3294B0120
:1020A0005C01E0E2F0E0E01BF10BA5E5B0E0AC0183
:1020B0009B010E94F3296B017C019F01DF010E94BB
:1020C00014299B01AC010E94FE299B01AC01280D43
:1020D000391D4A1D5B1DC701B6010E94062AF22E5A
:1020E000822F90E039E23F15D8F143E0249F900120
:1020F000112435952795122F109596ECC92E91E055
:10210000D92E00E085E5E82EEF188E2D01FD8F2DEC
:102110009601412F609160040E941A070F5F53E0FF
:10212000C50ED11C0C3389F70E941C0F9C8181E0E5
:10213000992319F0903219F48FEF80931101809157
:102140001101890F8C83DF91CF911F910F91FF9027
:10215000EF90DF90CF90BF90AF909F908F900895B9
:1021600025E530E0A901481B590BCA019A01220F4D
:10217000331F280F391F37FFBCCF2F5F3F4FB9CF19
:10218000EF92FF920F931F93CF93DF938C01C6ECD6
:10219000D1E0F12CE12CF8019481609160048091F0
:1021A0005F04FEE1EF16F104FCF49923F9F09E01BF
:1021B000409161040E941A072FEFE21AF20A239657
:1021C0008CE3E816F10439F70E941C0FF8018481B2
:1021D00090E00196817099278483DF91CF911F91C0
:1021E0000F91FF90EF900895992309F39E0140E02D
:1021F000E1CF90915E0490FF0CC0E6ECF1E08183AA
:1022000060834283339692E0EA37F907C1F70C9472
:102210001C0F08950F931F93CF93DF9300D00F925D
:10222000CDB7DEB78C018091C50181110AC09E0136
:102230002F5F3F4F42E36FEF0E941A078A8180931E
:10224000C501F8016481613069F08091C50140E009
:10225000662361F040E0623011F44091C50180E0F6
:1022600060E004C06091C50140E080E00E94F91088
:10227000F801848190E0019663E070E00E94F32809
:1022800084830F900F900F90DF91CF911F910F914A
:102290000895CF93DF9300D00F92CDB7DEB7909122
:1022A0005E0490FF0AC09E012F5F3F4F0E941A07F5
:1022B0004B8169818A810E94F9100F900F900F90D5
:1022C000DF91CF910895CF93DF93EC01EC81F0E0A3
:1022D000E158FC4F4491EEE5F4E0628181810E9477
:1022E00049118C818F5F8C83DF91CF910895CF93BB
:1022F000DF93EC01EEE5F4E0438162818C810E9482
:1023000049118C818F5F8C83DF91CF9108956F92FB
:102310007F929F92AF92BF92CF92DF92EF92FF9205
:102320000F931F93CF93DF9399E7E92E91E0F92E56
:10233000D0E0C0E010E0CC24C394D12C35E3A32E30
:1023400034E0B32ED7018D917D01F894E82FE2950A
:10235000EF70F0E021A18F70A60102C0440F551F5D
:102360008A95E2F7CA01922F982B91A392A18095AA
:10237000892382A3789400C0A6010C2E02C0440FCA
:10238000551F0A94E2F7BA0160957095E9E2F4E00E
:1023900088E8682E81E0782E00E021913191D30108
:1023A0009D903D01892D82958F7090E0DC01909683
:1023B0008C9190E0B92DBF7002C095958795BA9524
:1023C000E2F780FD67C0C901842B952B28173907D8
:1023D00039F09F0122503109D9018D939C9301E07E
:1023E000AE16BF06D1F6F701319780810E940D0A23
:1023F000CE3019F0E0EAEA95F1F7102B2196CF30B4
:10240000D10509F09FCF112309F448C081E08093E2
:10241000C2010E942E059093C1018093C00180915A
:10242000C0019091C1010E941F050697D8F18091CB
:10243000290490912A04909364048093630480910A
:102440002B0490912C0490936604809365048091F2
:102450002D0490912E0490936804809367048091DA
:102460002F049091300490936A04809369048091C2
:1024700031049091320490936C0480936B048091AA
:1024800033049091340490936E0480936D04109201
:10249000C20108C0C9018623972398CF8091C20149
:1024A0008111BDCF812FDF91CF911F910F91FF90AF
:1024B000EF90DF90CF90BF90AF909F907F906F9004
:1024C0000895AF92BF92CF92DF92EF92FF920F9357
:1024D0001F93CF93DF93EC018AE0A82E288122235B
:1024E00009F48CC02130C9F599818A81913021F499
:1024F00022960E949B0E05C0923029F422960E94DB
:10250000E60D2196EBCF933021F422960E94060926
:10251000F8CF943011F02196F4CF229630E020E0ED
:10252000AE014F5F5F4F8053990B8A30910550F099
:102530002150310930F38FE99FE00197F1F700C096
:102540000000F6CFA29EB001A39E700D11249C0145
:10255000260F371F8981EA01E3CFE22FF0E0E65032
:10256000FE4FB490822F86958695869590E0FC016B
:10257000E651FE4FE4902770F12C022E02C0F59434
:10258000E7940A94E2F731E0E322FF24FC01E652EB
:10259000FE4FC490D12C022E02C0D594C7940A9449
:1025A000E2F731E0C322DD24FC01E653FE4F049143
:1025B00010E002C0159507952A95E2F701701127E2
:1025C000E114F10419F081EE0E94E60DC114D1046A
:1025D00019F086EE0E94E60D8B2D0E949B0ECD28F1
:1025E00019F086EE0E940609EF2819F081EE0E948C
:1025F0000609012B09F485CF8CE27BCFDF91CF91C7
:102600001F910F91FF90EF90DF90CF90BF90AF9010
:1026100008954F925F926F927F928F929F92AF92A6
:10262000BF92CF92DF92EF92FF920F931F93CF93BF
:10263000DF93FC016280448081E08483EFE7F3E074
:102640007490EEEFF3E0E491CAE7D2E036ECE32ECB
:1026500031E0F32E46EAC42E43E0D42E52E0A52EFC
:10266000BB24B39488248A94912C55245A94E71956
:102670000E2F10E082E0861530F080915F04888391
:10268000809160048983411021C01B821A829701C6
:102690004A81698188810E941A07259683E0E80EA5
:1026A000F11CCC16DD0631F7DF91CF911F910F9110
:1026B000FF90EF90DF90CF90BF90AF909F908F9062
:1026C0007F906F905F904F900C941C0F8B818823AC
:1026D000E9F081508B83859DC00111246C8170E0ED
:1026E0000E94DF28FB01FF27E158FC4F8491E82F6F
:1026F000E719E59DC0011124B8010E94DF288091EF
:102700006104689FB00111247A83C1CF0E946F29B0
:1027100020916104269521582A9DA0012B9D500DE2
:102720001124452F5527841795070CF0B0CF82E070
:10273000861588F40E946F29B4010E94F3288883CB
:102740000E946F29209160042695622F70E00E94FC
:10275000F328280F29831A8280916104893C20F094
:1027600088EC8C838B8393CF8431D8F784E1F9CFC5
:1027700090E080E00E949A2921E08B3E9E4F09F074
:1027800020E0822F08956BEE7EEF90E080E00E94C3
:10279000BE2960E082E090E00E94A02960E083E032
:1027A00090E00E94A0291092250410922604109215
:1027B00027041092280460E084E090E00E94A029A1
:1027C00060E081E290E00E94A02960E085E090E076
:1027D0000E94A02960E086E090E00E94A0296FEFAF
:1027E00087E090E00E94A02940E050E0BA0188E034
:1027F00090E00E94B22960E08DE090E00E94A02964
:1028000040E050E0BA0188E190E00E94B22960E027
:1028100087E190E00E94A02940E050E0BA018CE1FD
:1028200090E00E94B22960E080E290E00E94A0293E
:1028300040E050E0BA0188E190E00E94B22940E017
:1028400050E0BA018FE090E00E94B22940E050E0F1
:10285000BA0183E190E00C94B2290E94B81381116F
:1028600002C00E94C31386E090E00E948C298093EE
:102870005B04803220F08770886180935B049091C4
:102880005B04892F817090FF04C0892F86958695FF
:1028900086950C948F06CF92DF92EF92FF926B0198
:1028A0007C010E940407B701A60188E090E0FF9038
:1028B000EF90DF90CF900C94B2295F926F927F924D
:1028C0008F929F92AF92BF92CF92DF92EF92FF9240
:1028D0000F931F93CF93DF9300D00F92CDB7DEB746
:1028E000182F762E042F622E90915E0490FF29C03F
:1028F000E92FE695AE2FB0E0A35EBE4F8C9180939A
:102900005C049E7F923081F59E012F5F3F4F812FA7
:102910000E941A074B8169818A810E94F9101093E5
:102920005F047092600400936104662051F060912E
:102930005E0470915F0480916004909161040E9434
:102940004B140F900F900F90DF91CF911F910F912B
:10295000FF90EF90DF90CF90BF90AF909F908F90BF
:102960007F906F905F900895823019F40091610418
:10297000D6CF863019F410915F04D1CF8930D9F3C6
:10298000893169F6E9518E2F8170582EE695F0E075
:10299000E658FC4FA590B490BB2486ECE82E81E06D
:1029A000F82ED12CC12C9CE3892E912CC601B401A8
:1029B0000E94DF28812F511013C0860F9701402FEE
:1029C000672D0E941A07CA0CDB1C83E0E80EF11C7D
:1029D0008AE7E81682E0F80649F70E941C0F9FCFAD
:1029E000861BECCFEEE5F4E0438128E0421B08F4BF
:1029F00040E021E0628181810C945D14EEE5F4E019
:102A0000438128E0420F08F44FEF21E06281818189
:102A10000C945D14EEE5F4E0628128E0621B08F49A
:102A200060E021E0438181810C945D14EEE5F4E0E7
:102A3000628128E0620F08F46FEF21E04381818119
:102A40000C945D14EEE5F4E0818121E04381628124
:102A500088500C945D14EEE5F4E0818121E043811F
:102A60006281885F0C945D1480916204882319F060
:102A700081508093620460915E0470915F04809144
:102A80006004909161040C944B1480916204833033
:102A900018F48F5F8093620460915E0470915F040C
:102AA00080916004909161040C944B14EEE5F4E085
:102AB00083E0808311828FEF828382E38383148299
:102AC00060817181828193810C944B141092230454
:102AD00080911C01E2EAF1E0882359F080913504ED
:102AE00087FF07C08EE1DF011D928A95E9F70C94FC
:102AF000DA0786E0F8CF1F93CF93DF93CDB7DEB729
:102B0000AA970FB6F894DEBF0FBECDBF8AE994E056
:102B10002091F100DC012D93CD01B4E0823A9B07B6
:102B2000B9F780919B04833009F471C0B8F4813007
:102B300009F448C0823009F4B2C08091E80083FFF4
:102B40003AC180919A0490919B049A3008F033C165
:102B5000E92FF0E0E95BF54D0C9407298A3009F480
:102B60008DC08B3009F470C0893039F780919A0498
:102B7000813219F780919E0490919F04009711F083
:102B80000297D9F68091E800877F8093E8008091D2
:102B9000E80082FF37C09091F3008091F200029725
:102BA00029F48091F1008B7F813021F48091F10034
:102BB000809375048091E8008B778093E8000E94F1
:102BC0000904BBCF80919A04813A09F0B6CF809175
:102BD000E800877F8093E80080919E0490919F0495
:102BE000892B61F460E286E794E070E00E94BB0408
:102BF0008091E8008B778093E8009FCF60E090E0C1
:102C000080E0F3CF809198048111C1CF96CF80915D
:102C10009A04813A09F091CF80919E0490919F048B
:102C2000892B09F08ACF8091E800877F8093E800A4
:102C30008091E80080FFFCCF80911C018093F1001F
:102C40008091E8008E77B9CF80919A04813209F0A3
:102C500074CF80919E0490919F04892B09F06DCFD1
:102C60008091E800877F8093E8000E9409048091AA
:102C70009C0480931C010E9466155FCF80919A048A
:102C8000813209F05ACF8091E800877F8093E80075
:102C90000E94090480919D04809374044ECF80911A
:102CA0009A04813A09F049CF8091E800877F8093A8
:102CB000E8008091E80080FFFCCF80917404BECFD3
:102CC000803899F0823809F076C080919E048F7028
:102CD000873008F070C08093E9008091EB0085FB9D
:102CE000882780F91092E90006C08091960490919F
:102CF0009704911182609091E800977F9093E8008B
:102D00008093F1001092F1008091E8008E77C0C1AD
:102D1000882309F4ADC1823009F04DC080919C0434
:102D20008111B1C180919E048F702FEF280F263042
:102D300008F041C08093E9002091EB0020FFA3C17F
:102D4000933031F48091EB0080628093EB009BC163
:102D50009091EB0090619093EB0021E030E001C096
:102D6000220F8A95EAF72093EA001092EA008091F8
:102D7000EB008860EACF81111EC010919C041F7780
:102D80008091E3008078812B8093E3008091E800BC
:102D9000877F8093E8000E9409048091E80080FF0B
:102DA000FCCF8091E30080688093E30082E0111102
:102DB00083E0809398048091E80083FF0AC08091AB
:102DC000E800877F8093E8008091EB008062809329
:102DD000EB00AA960FB6F894DEBF0FBECDBFDF9111
:102DE000CF911F9108958058823028F720919C043C
:102DF00030919D042C3DE3E03E07A1F583E08A83FA
:102E00008AE289834FB7F894DE01139620E03EE012
:102E100051E2E32FF0E050935700E49120FF03C00C
:102E2000E295EF703F5FEF708E2F90E0EA30C0F0D8
:102E3000C7968D939D932F5F243159F74FBF809193
:102E4000E800877F8093E8006AE270E0CE01019697
:102E50000E94BB048091E8008B778093E800ABCFA1
:102E6000C096E7CF80919E0490919F04432F5527F1
:102E70004330510509F44AC078F54130510509F451
:102E800085C08BE590E0ECEFF5E04230510509F0AC
:102E900092CF2091E800277F2093E8002091A004A2
:102EA0003091A1048217930708F49C0140E021159A
:102EB000310509F070C041116EC08091E80082FDBB
:102EC000C9CF80919804882329F2853019F2809126
:102ED000E80083FFF2CFBECF4132510509F447C06D
:102EE0004232510509F067CF8330910508F063CF76
:102EF000FC01EE0FFF1FEF56FE4F0190F081E02D19
:102F000082579E4FDC018C9190E01DC03327213009
:102F10003105E9F02115310579F022303105F9F05C
:102F20002330310509F047CFE9E6F6E0E4918E2F32
:102F300090E0E9E6F6E007C0E7E8F6E0E4918E2FDE
:102F400090E0E7E8F6E0009709F435CFA2CFEFE78D
:102F5000F6E0E4918E2F90E0EFE7F6E0F4CFEFE6B5
:102F6000F6E0E4918E2F90E0EFE6F6E0ECCF8330D0
:102F7000910508F020CF880F991FFC01E956FE4FFC
:102F80000190F081E02D89E090E083CF82E190E034
:102F9000E7E5F6E07ECF80919804882309F45ACFC4
:102FA000853009F457CF8091E80083FD53CF80919D
:102FB000E80082FD82CF8091E80080FF78CF909179
:102FC000F3008091F2002115310519F08830910548
:102FD00050F041E0089709F040E08091E8008E77DA
:102FE0008093E80064CF44914093F10031962150E2
:102FF00031090196E8CF803809F0DDCE8091E800F4
:10300000877F8093E800809199048093F1007CCEC3
:103010008111D1CE10919C04123008F0CCCE809159
:10302000E800877F8093E800109399040E940904C8
:10303000112311F084E005C08091E30087FDFACFF1
:1030400081E08093980442E061EC81E00E942804D2
:1030500042E261EC84E00E94280442E261EC82E0FA
:103060000E94280442E260EC83E00E942804A3CE80
:1030700080919C04813009F09ECE81E0933009F06C
:1030800080E0809397041092E9008091E800877FA8
:103090008093E8000E9409048ECE90915E0490FF18
:1030A0003DC09170811129C0926090935E046623A7
:1030B00051F060915E0470915F0480916004909182
:1030C00061040E944B1460915E04669570E04BE0D1
:1030D00050E084E091E00E947F29892BA9F01092B2
:1030E0005D0481E080933E0420E0409161046091A2
:1030F000600480915F040C945D148B3210F0946531
:10310000D4CF880F982BD1CF81E080935D040E94AB
:103110002E0590933C0480933B04E3CF0895809167
:103120005E048695815009F48AE261E00C944D18A2
:1031300080915E0486958F5F8B3208F081E061E0BC
:103140000C944D1890915E0490FF07C096959817C7
:1031500020F0961710F40C94981861E00C944D1818
:103160004F925F926F927F928F929F92AF92BF9297
:10317000CF92DF92EF92FF920F931F93CF93DF9343
:1031800000D000D00F92CDB7DEB77C01FC01838167
:103190009481892B31F08081918189238F3F09F0BF
:1031A000C6C50F900F900F900F900F90DF91CF91A9
:1031B0001F910F91FF90EF90DF90CF90BF90AF9055
:1031C0009F908F907F906F905F904F9008950E9496
:1031D000410C182F682F89819A810E940C06698101
:1031E0007A81812F0E94AA0A8C01F701928199238A
:1031F00009F472C5980122513F452031310508F08C
:1032000032C58FEF93E00E948C294EEED42ED00E63
:1032100006EF12E08823D1F080912004877009F432
:10322000C0CFF7018281882309F4BBCF82E00E94DE
:103230004008B7CF0115F4E01F0771F3C8010E94E1
:103240008C29811101C0DA940F5F1F4FD110F2CF8A
:1032500019821A821B821C82CC24CA9448012FEF47
:10326000821A920AC8010E948C2989831A828823B3
:1032700099F2813009F047C0580132E0A30EB11C29
:10328000C4010E948C29982E8A83882329F2C501C3
:103290000E948C29D82E8FEF890D833068F4580155
:1032A00043E0A40EB11CDB82DD2021F0CE010196AB
:1032B0000E9461128501D2CF54E09512FBCF5801D4
:1032C00084E0A80EB11CC80103960E948C29DD2061
:1032D00009F4A2CF882309F49FCF8150990BC89E8F
:1032E0009001C99E300D1124ED2DE150FF0BCF014F
:1032F000820F931F0197F0F2EFE9FFE03197F1F7AA
:1033000000C00000F7CFCE0101960E946112540167
:10331000D1CF81E00E9458080E9401087DCF81E052
:103320000E941D08F9CF82E0F5CF82E0F9CF0F3B74
:103330008CE5180709F44AC098F1003CFCE51F072A
:1033400009F0ADC490915B04892F8695869586958A
:103350008F5F8F719770843008F059C0880F880F85
:10336000880F892B80935B0480915B0410C083E0FD
:103370000E94E90680915B040E94B10C4DCF8091C0
:103380005B04982F987FE9F1885080935B04887FD5
:1033900091E009F490E080915B0490FB80F913C008
:1033A00080915B04982F969596959695933040F46E
:1033B0009F5F990F990F990F8770892B80935B04FA
:1033C00080915B04816080935B0419C080915B04F1
:1033D00080FF09C08E7F80935B040E94B10C80E067
:1033E0000E948F0619CF80FD17CF816080935B0408
:1033F000813019F489E080935B0480915B040E9422
:10340000B10C80915B04869586958695E9CF909363
:103410005B04AACF27E245EE65EE5AC426E241EEF0
:1034200060EE56C427E245EE64EE52C426E241EE59
:1034300062EE4EC428E241E0EFCF80913504806116
:1034400006304CE5140709F489C080913504886082
:1034500007301C4508F482C08091350480627EC02C
:103460000C308CE5180709F48EC070F48091350497
:103470008C600A30ECE51E0709F470C008F47DC0CA
:10348000809135048E7F6AC080913504877F0E302D
:103490002CE5120709F462C0809135048B7F0F3050
:1034A0001C4508F45BC0809135048F7E57C00B3FEC
:1034B0004CE5140709F459C030F503318CE51807C1
:1034C00009F46DC078F40131ECE51E0709F463C01E
:1034D00002311C4509F08DC40E94661580913504A7
:1034E0008F773CC005312CE5120709F460C008F461
:1034F00074C08091360481600A3F1C4509F079C48C
:103500008093360476C40F3F5CE5150709F44BC081
:1035100088F4809136048D7F0D3F9CE5190781F377
:10352000809136048E7F0E3F1C4550F38091360407
:103530008360E6CF0130FDE51F0709F457C008F4AA
:1035400042C060E002301D4509F053C48EE090E0B7
:103550000E94A0294EC48091350481608093350477
:1035600048C4809135048460F9CF8091360482602C
:10357000C7CF809135048064F1CF0E946615809199
:1035800035048068EBCF809135048D7FE7CF809143
:1035900035048F7DE3CF809135048F7BDFCF809121
:1035A0003504837FDBCF809136048C7FA9CF809157
:1035B000350482FB992790F921E0922790FB82F94C
:1035C00090FB83F9CBCF80913604982F9095917022
:1035D0008E7F892B90FB81F993CF0E946615909185
:1035E0003504892F97FB87F98058B8CF61E0AECFBB
:1035F0008091230406314CE5140709F0A9C38A7AA7
:1036000091E009F490E09093AA03811106C089E249
:103610000E94B0050E944005FFCD85E3F9CF85E308
:1036200083C380915E0480FF1BC08E7F80935E0405
:1036300060915E0470915F048091600490916104D8
:103640000E944B1410925D045FEF80E792E05150AE
:1036500080409040E1F700C000000E941C0FDCCDCC
:10366000816080935E0461E086950E944D18D4CD00
:103670004FE858E168E978E10E94FF06CDCD48E9BE
:1036800058E16FE878E1F8CF42E255E16BE275E18D
:10369000F3CF4BE255E162E275E1EECF4AE055E14E
:1036A00066E175E1E9CF46E155E16AE075E1E4CF15
:1036B00042EF54E16EEF74E1DFCF4EEF54E162EF81
:1036C00074E1DACF44E355E165E475E1D5CF45E433
:1036D00055E164E375E1D0CF61E081E0C6CF65E0FC
:1036E00082E00E94A21898CD68E086E0FACF6EE0F2
:1036F00089E0F7CF64E18FE0F4CF67E185E1F1CFB6
:1037000061E088E1B2CF62E289E1EBCF61E083E280
:10371000ACCF0115ECE51E0709F445C00E3D1C4574
:1037200009F44EC0F70100811181992309F44BC0BF
:10373000C8010E94410CD82E682FC8010E940C06B7
:10374000B8018D2D0E94B70A8C01882EF701D28016
:10375000A580A2943FE0A322809120048770A1F06D
:10376000CD2CDD2091F0812F807F803421F080E20C
:10377000800F883048F082E00E9440088091200449
:103780008770CC24C3948111C12CB12EB2942FE048
:10379000B222FBE0FB1508F450C0EB2DF0E0EF5A2D
:1037A000F54D0C9407290E9466152FEF34E34CE089
:1037B000215030404040E1F700C000000E94C20D9F
:1037C0000E94C31329CDC8010E94E405D82EB8CFAA
:1037D000212F2F70A22E107F19F0A29490EFA92212
:1037E000DD20C9F0AA2069F080E2800F883010F057
:1037F00081100BC080912304A82AA09223040E9468
:103800004005802F0E94E60D18C080912204A82A4E
:10381000A0922204F4CF802F0E940609AA2069F00A
:10382000A094005E083010F081102AC0809123041B
:10383000A822A09223040E9440052B2D2850330B70
:103840002430310520F40E9483060E94670ACC20B0
:1038500009F4A7CC8091200480FDA3CCF70112824B
:103860008595859585950E945808C7010E94B018D6
:10387000809120048595859585950E941D0891CCA1
:1038800080912204A822A0922204D5CF312F3F702C
:10389000932E107F103219F0929480EF9822882096
:1038A00071F041E0841661F1DD20B9F1AA2071F1D7
:1038B000F701858180FFA5CF8F70858327C0DD202C
:1038C00091F090912404892D892BA11003C00E94AE
:1038D0004D06B3CF51E0A512FACF981709F4ADCF3A
:1038E00080932404AACFA11006C00E943A05892D16
:1038F0000E944206A2CF81E0A81609F49ECFF5CF20
:10390000DD2031F095E09A1508F497CF892DDFCFAF
:10391000E4E0EA1508F491CFEACFAA2041F3F9E3F5
:103920008F1209C02FEF37EE43E021503040404066
:10393000E1F700C00000802F0E9406097ECF812F92
:1039400086958695837061F0813009F076CFC80145
:103950009370D11002C090E080E00E9457066DCFB6
:10396000C8019370D11002C090E080E00E946D0603
:1039700064CF802FDD2039F00E94A5090E94B30793
:103980000E94B3075ACF0E948308FACF812F837019
:1039900009F066C0D11051CF802F8295869587702F
:1039A000880F880F602F6F70462E512C712C612C60
:1039B000082E04C0440C551C661C771C0A94D2F7D0
:1039C00040E050E0BA0104FF0FC04FE050E060E07B
:1039D00070E004C0440F551F661F771F8A95D2F709
:1039E0004095509560957095812F8695869583704A
:1039F000823019F1D8F40091250410912604209109
:103A0000270430912804813069F04429552966291A
:103A10007729CB01BA0160237123822393230E946B
:103A200079080BCF402A512A622A732ACB01BA01A6
:103A30006429752986299729F2CF442955296629B1
:103A400077290091250410912604209127043091B4
:103A50002804CB01BA016027712782279327DFCF83
:103A60008695DD2011F0812F8170882309F4E5CE41
:103A7000802F829586958770880F880F602F6F70D2
:103A8000462E512C712C612C082E04C0440C551C60
:103A9000661C771C0A94D2F740E050E0BA0104FF9C
:103AA0000FC04FE050E060E070E004C0440F551FCD
:103AB000661F771F8A95D2F740955095609570954F
:103AC000812F869586958370823019F1D8F4009104
:103AD000A5041091A6042091A7043091A804813078
:103AE00069F04429552966297729CB01BA01602359
:103AF0007123822393230E94F7079FCE402A512AE5
:103B0000622A732ACB01BA0164297529862997296B
:103B1000F2CF44295529662977290091A5041091EF
:103B2000A6042091A7043091A804CB01BA01602714
:103B3000712782279327DFCF1F70DD2029F0812F87
:103B40000E945808802FC3CE802F0E944206812FEA
:103B50000E941D0872CE802F52EF851609F450C0C6
:103B6000581578F090EF891619F1E1EF8E1609F4E7
:103B70003FC0DD2009F467C0A11043CE812F8F71B3
:103B80003CC0F3EF8F1609F440C024EF8212F1CF4E
:103B9000DD2009F44DC01F71812F0E94580858E0A4
:103BA000159FC0011124836080932004812F25C0BC
:103BB000DD20C9F034E03A1508F43FCE1F7161E012
:103BC00070E080E090E004C0660F771F881F991FA7
:103BD0001A95D2F70091A5041091A6042091A7048C
:103BE0003091A804A4CF45E04A1508F426CEE6CFCC
:103BF000812F8F71DD2009F4ABCF0E9458081DCEB4
:103C0000812F8F71DD20C9F3A3CF60E070E0CB017D
:103C1000DD2009F470CF1F7161E070E080E090E07A
:103C200004C0660F771F881F991F1A95D2F763CFBC
:103C300081E00E94400881E08A1508F0FECD82E014
:103C40000E944008FACDAA2059F0893309F073CEBA
:103C50009FEFE7EEF3E09150E040F040E1F769CEEE
:103C6000812F8F7175CF0031FFE51F0709F451CB0C
:103C700001312FE5120709F456CB0D3B2CE5120755
:103C800009F47DCB08F053CB0B3B4CE5140709F44A
:103C90006ECB80E00C3B5CE5150709F469CB033F74
:103CA0002CE5120709F4BACB08F05EC0083D4CE5DC
:103CB000140709F4AFCB093D5CE5150709F4BACB4D
:103CC000073D8CE5180709F05BC026E241EE61EE86
:103CD000C7010E94B80EA0CA00313FE5130709F4DE
:103CE0001ECB01314FE5140709F41FCB033F3CE520
:103CF000130709F493CB08F08CC0083D5CE5150769
:103D000009F488CB093D8CE5180709F493CB073DEE
:103D1000ECE51E07D1F206311C4509F003CD809178
:103D2000AA0381117CCC89E20E94850573CC85E0D1
:103D3000DE01119601900D928A95E1F7F70122813B
:103D400089819A81211143CA0E94E405182F47CA2C
:103D50008272F801E25CFC45E431F10508F0D9CC4F
:103D6000E35AF54D0C940729053FECE51E0709F4CD
:103D70005DCB08F457CB063F2CE5120709F455C07C
:103D80001092A40402302CE5120708F431CC06315D
:103D90003CE5130738F098012A5F3C45293031058E
:103DA00008F026CC0E946D0A909336048093350467
:103DB00000314CE5140709F4EACB08F078CB083061
:103DC0008CE5180709F4D5CB08F04ACB0430ECE5B4
:103DD0001E0709F4C6CB08F030CB02302CE51207E1
:103DE00009F4B9CB80913504826003301C4509F495
:103DF000B5CB609135041091360484E090E00E94C8
:103E0000A029612F81E290E00E94A0290E946615FE
:103E100003CA053FFCE51F0709F408CB08F402CBF1
:103E2000063F3CE5130709F076CF27E245EE66EE44
:103E30004FCF1F93CF93DF938091B103807FA9F47D
:103E40008091AE03882389F08091E303D091B2037F
:103E50006091AC037091AD03A091AF03B091B0033A
:103E6000C62FC72316E0D81304C0DF91CF911F914E
:103E7000089590E0109711F0CF3F19F401968770E4
:103E8000F2CF189F9001199F300D1124F901ED54C4
:103E9000FC4F41814713F2CF40814613EFCF42815F
:103EA0004111ECCF438154814A1B5B0B483C5105C7
:103EB00028F78091B1038F7080618093B103F9017D
:103EC000E854FC4F80818F70806180838CEA93E09E
:103ED0000E94B018DF91CF911F910C943806AF92D9
:103EE000BF92CF92DF92EF92FF920F931F93CF93E7
:103EF000DF93CDB7DEB761970FB6F894DEBF0FBE84
:103F0000CDBF8C0185E0F801DE011D9601900D9278
:103F10008A95E1F7F80180819181E2802CEAA22E56
:103F200023E0B22E6091AF037091B003611571056B
:103F300009F43EC13091AC034091AD03232F2423FB
:103F40002F3F09F435C1C380D480F090AE03F60151
:103F5000E61BF70BFF2009F4FBC02091B103522FA1
:103F6000507FE83CF10508F0BBC0511178C0FE2C31
:103F7000491321C038131FC0E1101DC02F702061EC
:103F80002093B103C5010E94B0188091B103F801DC
:103F900085838F2D61960FB6F894DEBF0FBECDBF1F
:103FA000DF91CF911F910F91FF90EF90DF90CF9015
:103FB000BF90AF900895CD2829F0282F29232F3FB7
:103FC00009F014C120E0F22FF170DF2E20FF3DC078
:103FD0002091E3034091B20356E0241315C08D876E
:103FE0009E878D859E850E94830C292F22952F7098
:103FF0002230F8F0243020F59F70F9F0F801958117
:10400000907FD9F4D12C1FC030E0529FF001539F14
:10401000F00D1124ED54FC4F6181961306C06081B0
:10402000861303C06281E61210C02F5F3F4F2770D6
:10403000D4CF9F7011F0882329F3805E883010F36D
:10404000C8010E94B018FD2CA4CFEE2009F4A1CF26
:104050008091B10381608093B103F12C9ACF491311
:1040600012C0381310C0E1100EC0F8012583C8013A
:104070000E94B01886E0F801ACEAB3E001900D921E
:104080008A95E1F786CF8D879E878D859E850E94D4
:104090008D0C882309F1EE20F9F08091B103803274
:1040A00070F02091AC033091AD0338872F831986CF
:1040B000DB86CA868C87CE0107960E94B01886E000
:1040C000F801ACEAB3E001900D928A95E1F70E9405
:1040D000191FFF24F3945DCFC8010E94B018F9CFD7
:1040E00051110AC08CEA93E00E94B01886E0F501F5
:1040F00011928A95E9F7B1CF49130FC038130DC05B
:10410000E1100BC0F8012583C8010E94B01886E0B9
:10411000F50111928A95E9F73CCF8D879E878D85B1
:104120009E850E948D0C8823B9F2EE20A9F2809121
:10413000B103803220F22091AC033091AD033A8379
:1041400029831B82DD82CC828E83CE010196B5CF7E
:10415000E83CF105E0F6FE2CEE2009F4BDCF491352
:1041600016C0381314C08091B10380FD83CF982FFF
:10417000907F09F47FCFF8018583903F09F477CFD2
:10418000982F907F905F8F70892B858370CF8D875C
:104190009E878D859E850E948D0C811190CF809188
:1041A000B10381608093B103C8010E94B018F1CEC1
:1041B000EE2009F491CF8D879E878D859E850E9484
:1041C0008D0CF82E882309F487CF86E0F801ACEA3D
:1041D000B3E001900D928A95E1F78091AC03909144
:1041E000AD030E94830C0E94191FD3CE21E02E251F
:1041F000EACE1F93CF93DF93CDB7DEB767970FB6A5
:10420000F894DEBF0FBECDBF342F4B8B252F5C8BB8
:104210006D8B7E8B8F8B8E899F896111109222040A
:104220001A8A198A3D872E876F87998B888B86E03B
:10423000FE013D96DE01179601900D928A95E1F7F9
:10424000CE0107960E946F1F882389F016E08091A7
:10425000E3039091B203891349C067960FB6F894AF
:10426000DEBF0FBECDBFDF91CF911F91089586E0D5
:10427000FE013796DE01119601900D928A95E1F7C5
:104280008A859B85892B11F38F81988589238F3FA0
:10429000E9F22091B20330E0C901019687709927B5
:1042A0004091E3034817190671F40E9466151092B5
:1042B000B2031092E30386E0ECEAF3E0DF011D9223
:1042C0008A95E9F7C3CF96E0929FD001939FB00DF6
:1042D0001124AD54BC4FFE01319601900D929A9578
:1042E000E1F78093B2030E943806B0CF819FC001EE
:1042F00011248D549C4F0E946F1F882309F4ADCF69
:104300008091E30390E00196877099278093E303FF
:104310009ECF1F920F920FB60F9211242F933F93AF
:104320004F935F936F937F938F939F93AF93BF93BD
:10433000CF93DF93EF93FF93D091E900DF708091EB
:10434000EC00C82FC17080FDC0E81092E900809198
:10435000F000877F8093F00078940E947B15109284
:10436000E9008091F00088608093F000CD2BCF7041
:10437000C093E900FF91EF91DF91CF91BF91AF9191
:104380009F918F917F916F915F914F913F912F916D
:104390000F900FBE0F901F9018951F920F920FB69F
:1043A0000F9211242F933F934F935F936F937F93BB
:1043B0008F939F93AF93BF93EF93FF938091E1000F
:1043C00082FF09C08091E20082FF05C08091E10078
:1043D0008B7F8093E1008091DA0080FF24C0809180
:1043E000D80080FF20C08091DA008E7F8093DA00B1
:1043F0008091D90080FF9BC080E189BD82E189BDA9
:1044000009B400FEFDCF81E080939804809173048D
:10441000811109C00E948F030E945A048091E2001A
:1044200084608093E2008091E10080FF17C080915A
:10443000E20080FF13C08091E2008E7F8093E20053
:104440008091E20080618093E2008091D8008062D8
:104450008093D80019BC85E0809398048091E10096
:1044600084FF29C08091E20084FF25C080E189BDDE
:1044700082E189BD89B5982F917080FFFBCF809133
:10448000D8008F7D8093D8008091E1008F7E80934B
:10449000E1008091E2008F7E8093E2008091E20053
:1044A00081608093E20080919904882309F445C0DB
:1044B00084E0809398048091E10083FF27C080917D
:1044C000E20083FF23C08091E100877F8093E100B9
:1044D00082E080939804109299048091E1008E7F8D
:1044E0008093E1008091E2008E7F8093E2008091D2
:1044F000E20080618093E20042E060E080E00E94A0
:1045000028048091F00088608093F000FF91EF9183
:10451000BF91AF919F918F917F916F915F914F91DB
:104520003F912F910F900FBE0F901F90189519BCBF
:10453000109298041092730476CF8091E30087FD67
:1045400093E090939804B7CFCDB7DEB7AA970FB694
:10455000F894DEBF0FBECDBF84B7877F84BF0FB690
:10456000F894A89580916000886180936000109213
:1045700060000FBE80E890E00FB6F8948093610071
:10458000909361000FBE85B7806885BF85B780684E
:1045900085BF8AE195E090939F0180939E010E94E0
:1045A0008F030E945A048091E20084608093E200AD
:1045B0007894809198048823A1F01091E9001F70ED
:1045C0009091EC00892F817090FD80E8182B10925B
:1045D000E9008091E80083FD0E947B151F70109315
:1045E000E90082E084BD93E095BD9AEF97BD80938A
:1045F0006E0009E711E0F80181918F010E940D0A18
:10460000F1E008381F07B9F786E60E940D0A80E33B
:104610000E940D0A81E30E940D0A82E30E940D0AA6
:1046200083E30E940D0A87E30E940D0AE9E2F4E0A9
:1046300085E394E0A3E6B4E0119211921D921D92DD
:104640008E179F07C9F70E9487112FEF46E781E079
:10465000215040408040E1F700C000000E948711D7
:104660008091630480FF17C06FEF82E290E00E94A8
:10467000A0296FEF83E290E00E94A0296FEF84E20F
:1046800090E00E94A0296FEF7FEF90E080E00E9411
:10469000BE290E94C20D0E94B813811102C00E945F
:1046A000C3133F9A479A269A2E9882E280938000FD
:1046B00089E1809381008FEF9FEF90938700809333
:1046C00086000E942D1482E290E00E948C298132A3
:1046D00009F0D4C483E290E00E948C29873009F06D
:1046E000CDC484E290E00E948C29873209F0C6C4D0
:1046F0000E94B813811102C00E94C31382E090E0AF
:104700000E948C2980934E040E946D0A9093360477
:104710008093350483E090E00E948C29682F70E03C
:1047200090E080E00E9479080E942D148091370467
:10473000811133C00E94B813811104C00E94C313B9
:104740000E94561588E090E00E94942960935E04D0
:1047500070935F0480936004909361046E7F71F4A2
:104760000E94561588E090E00E94942960935E04B0
:1047700070935F0480936004909361040E94040727
:1047800010925D0480915E0480FF04C060E0869515
:104790000E944D1881E08093370482E191E090936C
:1047A00039048093380458E1E52EF12C60E4B62EEC
:1047B0007FE6C72E74E0D72E8091980400E112E1C5
:1047C000853009F4C1C10E948711882359F08FB741
:1047D000F89440916F04509170046091710470914D
:1047E00072048FBFEFE4F4E0A3E6B4E010E000E071
:1047F000702F8D919D91219131912817390709F4DE
:10480000B7C12827392760E088248394912CA90117
:1048100048215921452B09F4A5C169A37AA39C011C
:104820002821392191E0232B09F490E09BA30E94D9
:104830002E058160782F9DA38CA349A15AA16BA15D
:104840008DA10E94F920000F111FF801E15BFB4FC1
:1048500080819181882699269182808280915D0451
:104860008823D1F180915C04E0915E04E695E81B19
:10487000E0933D04823009F092C1F0E0E850FA4F35
:10488000E4910E2F10E0F3E68F2EF1E19F2E809140
:104890003E04882361F010923E040E942E059093FE
:1048A0003C0480933B041092400410923F040E9409
:1048B0002E05E0913B04F0913C048E1B9F0B8F3F33
:1048C0009F4750F4E00FF11FF0933C04E0933B044A
:1048D0008BE394E0F401099586E0E7E4F4E0DE017F
:1048E000119601900D928A95E1F79090490480907D
:1048F0004A0410914B0400914C0410924904109208
:104900004A0410924B0410924C04892D882909F412
:1049100048C080914504909146040E941F059C0167
:1049200090914404992309F4D0C323333105C8F18D
:104930009F3F19F09F5F90934404992059F00E9483
:1049400085099FEF19140CF491E0899F802D1124A3
:1049500080934904882059F00E9485099FEF18141C
:104960000CF491E0899F802D112480934A043091AA
:1049700049043323B1F020914A04222391F045EBFE
:104980003403C0011124992309F475C1909349049B
:1049900045EB240390011124332309F470C13093B3
:1049A0004A04812F802B09F448C0809142049091E1
:1049B00043040E941F059C0190914104992309F42E
:1049C0007FC325363105C8F19F3F19F09F5F909353
:1049D0004104112359F00E9463099FEF11160CF452
:1049E00091E0899F802D112480934B04002359F07E
:1049F0000E9463099FEF10160CF491E0899F802DAF
:104A0000112480934C0430914B043323B1F0209156
:104A10004C04222391F045EB3403C0011124992367
:104A200009F431C190934B0445EB24039001112408
:104A3000332309F42CC130934C04809149049091A4
:104A40004A04892B90914B04892B90914C04892B1B
:104A500011F00E94B30786E0FE013196A7E4B4E0AE
:104A600001900D928A95E1F70E94830690914D0482
:104A7000891731F00E94830680934D040E94670AD3
:104A800080919804843009F097CE83E08093E90008
:104A90008091E80082FF90CE8091E80090E085FF51
:104AA00006C00E94AE03882309F4F5C091E080910E
:104AB000E8008B778093E800992309F47DCEE981A3
:104AC000E150E33108F069C1F0E0EF58F54D0C9486
:104AD000072980919804843039F180E00E948F0684
:104AE00080E00E94670A10923A040FB6F894A895E5
:104AF000E09260000FBEB092600083B7817F846057
:104B000083BF83B7816083BF7894889583B78E7F96
:104B100083BF0FB6F894A895809160008861809358
:104B20006000109260000FBE80919704882361F0AE
:104B30000E948711E3E6F4E081919191892B09F0BD
:104B400087C2CE16DF06C1F780919804853009F43C
:104B5000C0CF0E9466150E942D140E9483060E94F9
:104B6000670A31CE6F5F880C991C6F3009F04FCE09
:104B70000F5F1F4F0630110509F03ACE8FEF8EA35D
:104B80008FA318A60E942E058160782F9AA789A767
:104B90004EA15FA168A58AA50E94F9205FCE86304C
:104BA00059F4F0E0EB50FA4FE4910E2F10E0E7E7F4
:104BB0008E2EE1E19E2E6BCE893061F4E695F0E019
:104BC000EE50FA4FE4910E2F10E071E5872E7FE052
:104BD000972E5DCE8F3061F4E695F0E0E151FA4F0B
:104BE000E4910E2F10E06BE7862E6FE0962E4FCEED
:104BF000853159F4F0E0E451FA4FE4910E2F10E0C2
:104C000059EE852E5FE0952E42CE08E210E027E3B4
:104C1000822E20E1922E883109F439CE833249F474
:104C2000EAEEF5E0059114914AE0842E41E1942EDC
:104C30002ECE04EF11E090EC892E90E1992E843273
:104C400009F425CE853281F48E2F63E00E94C528B9
:104C5000E92FF0E0E951FA4FE4910E2F10E039E02E
:104C6000832E33E1932E13CE00ED17E089E1882ED9
:104C700085E0982E0CCE81E08093490489CE81E0B6
:104C800080934A048ECE81E080934B04CDCE81E0A8
:104C900080934C04D2CE00E210E0CE0101964C018C
:104CA0008091E80085FD0AC08091E8008B778093B1
:104CB000E8000E94AE03882399F3F8CE8091F100BA
:104CC000F40181934F010150110951F7EFCE1A827F
:104CD00089E08B831AC08A81823009F4E8C183306D
:104CE000D9F1813009F059C02FB7F89460916F0461
:104CF0007091700480917104909172042FBF0E9492
:104D00000D296B837C838D839E83809198048430EE
:104D100009F052CD1091E9001F709091EC00892F9D
:104D2000817090FD80E8182B82E08093E9008091EB
:104D3000E80080FF0DC050E040E060E270E0CE018E
:104D400001960E94DF038091E8008E778093E8004F
:104D50001F701093E90030CDDE011196E3E6F4E018
:104D600080819181329612969C93129713968C9320
:104D70001397129624E0EF36F20791F7C6CF8A8197
:104D8000823059F46B817C818D819E810E940D2936
:104D900085E290E00E94A029B8CF8FEF8983B5CF3C
:104DA0004C816B818A810E947B0A982789279827EA
:104DB0009E838D83AACF2D813E81322723273227E0
:104DC0004C816B818A810E94C60C9FCF0E94EF0CA0
:104DD0009CCF8A81893061F48B8143E0849FC0013C
:104DE00011246FEF70E00E94DF28862F0E94E906F1
:104DF0008A818138C1F060F4803809F086CF20E0E4
:104E00004B816091600480915F040E945D147DCFAE
:104E1000823859F1833809F078CF20E0409161045D
:104E20006C818B81F2CF60E08B810E944D189B8159
:104E300080915E04911111C08E7F80935E04109268
:104E40005D048FEF90E7E2E081509040E040E1F7B1
:104E500000C000000E941C0F58CF816080935E0448
:104E600060E086950E944D1850CF8B81809362043C
:104E70004CCF8A81893059F08A30C1F0813821F1D4
:104E8000B8F4803809F041CF8091610422CF80913D
:104E90005B04869586958695FFEF8F9FC001112450
:104EA00063E070E00E94DF286B832FCF1B822DCF41
:104EB000823891F0833809F028CF80915F048B838A
:104EC000809160048C8321CF80915E0480FF02C0BA
:104ED0008695FFCE80E0FDCE80916204FACE80916F
:104EE0005B040E94B10C60915E0470915F0480913C
:104EF0006004909161040E944B1407CF80E18A8383
:104F000004CF81E08A838AE0E4CE0C8110E00D3189
:104F1000110508F0FACE8A809B8098248924982471
:104F2000CE0101963C01080F191FC4018A509D4F04
:104F30006016710609F4E9CEFAE08F16F1E09F06DB
:104F400058F40E948C29F3018483FFEF8F1A9F0A83
:104F50002FEF621A720AE9CFF3011482F6CF8C8028
:104F6000912C4DE18416910408F0CFCE0A811B816B
:104F7000102701271027CE0101963C01800E911EBB
:104F8000C8018A509D4F8016910609F4BECE0A30A2
:104F9000E1E01E0720F4F30164810E94A029FFEFE5
:104FA0006F1A7F0A0F5F1F4FEBCF0E94B60CADCE7A
:104FB00084E0A5CF0C8110E00D31110508F0A5CEDD
:104FC0008A809B80982489249824CE0101963C01F4
:104FD000080F191FC40186960615170509F495CE0A
:104FE000F0ED8F16F2E09F0658F40E948C29F30131
:104FF0008483FFEF8F1A9F0A2FEF621A720AEACF9B
:10500000F3011482F6CF8C80912C4DE1841691042B
:1050100008F07BCE0A811B81102701271027CE01C3
:1050200001963C01800E911EC8018696801691065D
:1050300009F46BCE003DE2E01E0720F4F301648129
:105040000E94A029FFEF6F1A7F0A0F5F1F4FECCF5E
:1050500009BD19BD09B400FEFDCF8091D8008F7D38
:105060008093D8008091E00082608093E00080917E
:10507000E00081FDFCCF0E94661566CD60E085E210
:1050800090E00E94A0290E94EF0C0E94B60C61E201
:1050900082E290E00E94A02967E083E290E00E9413
:1050A000A02967E284E290E00E94A02921CB85E25A
:1050B00090E00E948C291B821C821D828E8325CE4B
:1050C0002D32314008F082CCB8CC2D32314008F07E
:1050D00031CC67CC78941F921FB61F9211248F9306
:1050E0009F93AF93BF9380916F0490917004A091B0
:1050F0007104B09172040196A11DB11D80936F04DB
:1051000090937004A0937104B0937204BF91AF9117
:105110009F918F911F901FBE1F9018951F921FB6D1
:105120001F9211248F939F93AF93BF9380913A0462
:10513000811113C080916F0490917004A09171044B
:10514000B09172044196A11DB11D80936F0490939C
:105150007004A0937104B0937204BF91AF919F91BA
:105160008F911F901FBE1F901895DB018F939F9307
:105170000E94F329BF91AF91A29F800D911DA39F23
:10518000900DB29F900D11240895991B79E004C0F1
:10519000991F961708F0961B881F7A95C9F7809576
:1051A000089587FB082E062687FD819567FD61958A
:1051B0000E94C5280EF4919507FC81950895AA1BBD
:1051C000BB1B51E107C0AA1FBB1FA617B70710F0F2
:1051D000A61BB70B881F991F5A95A9F78095909524
:1051E000BC01CD01089597FB072E16F4009407D05B
:1051F00077FD09D00E94DF2807FC05D03EF490958A
:1052000081959F4F0895709561957F4F0895EE0F9A
:10521000FF1F0590F491E02D0994692796276927CF
:1052200078278727782708950E94282A332312F4A5
:105230008A1B9B0B0C941E290E94282AB7FF0895F5
:10524000821B930B08958F929F92AF92BF92CF9241
:10525000DF92EF92FF92CF93DF93EC016881798127
:105260008A819B81611571058105910521F464E2B4
:1052700079ED8BE597E02DE133EF41E050E00E94BE
:10528000D42949015A019B01AC01A7EAB1E40E946B
:10529000F3296B017C01ACEEB4EFA50194010E94EF
:1052A000012ADC01CB018C0D9D1DAE1DBF1DB7FF7A
:1052B00003C00197A109B04888839983AA83BB835F
:1052C0009F77DF91CF91FF90EF90DF90CF90BF90CD
:1052D000AF909F908F9008950E942329089580E0B9
:1052E00091E00E9423290895B0E0A0E0809300019E
:1052F00090930101A0930201B09303010895FC0172
:105300004150504030F001900616D1F73197CF014F
:105310000895882799270895F999FECF92BD81BDF8
:10532000F89A992780B50895A6E1B0E044E050E0EE
:105330000C94C629A8E1B0E042E050E00C94C629E4
:10534000262FF999FECF92BD81BDF89A019700B43E
:10535000021639F01FBA20BD0FB6F894FA9AF99ADE
:105360000FBE08950396272F0E94A1290E94A0290D
:10537000252F0E94A129242F0C94A1290196272FC3
:105380000E94A1290C94A029DC01CB01FC01F99910
:10539000FECF06C0F2BDE1BDF89A319600B40D9281
:1053A00041505040B8F70895052E97FB1EF4009425
:1053B0000E94EB2957FD07D00E94062A07FC03D064
:1053C0004EF40C94EB2950954095309521953F4F24
:1053D0004F4F5F4F089590958095709561957F4FE1
:1053E0008F4F9F4F08950E94282AA59F900DB49F2C
:1053F000900DA49F800D911D11240895B7FF0C946A
:10540000F3290E94F329821B930B0895A1E21A2E1F
:10541000AA1BBB1BFD010DC0AA1FBB1FEE1FFF1F58
:10542000A217B307E407F50720F0A21BB30BE40BA8
:10543000F50B661F771F881F991F1A9469F76095EF
:105440007095809590959B01AC01BD01CF010895A9
:10545000A29FB001B39FC001A39F700D811D1124B5
:10546000911DB29F700D811D1124911D0895F89416
:10547000FFCF9C0C9C0CA50CA50CA70CA50CA50C97
:10548000A50C9C0C9C0CAC0CA50CA50CAC0C6016D3
:105490008816DB168816DB16BB16F316DB16FB1711
:1054A0000818E81BE81B461C461C9F1CB91C1D1C49
:1054B0001D1CC61C9C1DAB1DAB1D111B381B3F1BAF
:1054C000441B491B4E1B531B581B5D1B621B671B58
:1054D0006C1B6F1B741B771B7A1B7D1B801B831B34
:1054E000861B67266B26BF26D026DB26E626E92606
:1054F00039276F27CD26CD267E2781278527AF2701
:08550000D527D827DA2703287C
:105508000100000001191A1B1C1D1E1F2021220169
:1055180002011C05820D610D5D0D590D010001028E
:105528000202020606060909090909090F0F0F0FE9
:105538000F0F1515151819191919191919191919F4
:105548002324252525252525818283E200E900EAF3
:1055580000B500B600B700CD008301CC008A0192E7
:105568000194012102230224022502260227022A8D
:1055780002B300B4006F00700090919293959496D6
:105588009734F7F6F5F4F1F06630313233374022CC
:0E559800BC8A016801AC000E0627064706001B
:00000001FF
